:080000000C948C000C9400002C
:100008000C9400000C9400000C9400000C94000068
:100018000C9400000C9400000C9400000C94000058
:100028000C9400000C9400000C9400000C94000048
:100038000C9400000C9400000C9400000C94000038
:100048000C9400000C9400000C9400000C94000028
:100058000C9400000C9400000C9400000C94000018
:100068000C9400000C9400000C9400000C94000008
:100078000C9400000C9400000C9400000C940000F8
:100088000C9400000C9400000C9400000C940000E8
:100098000C9400000C9400000C9400000C940000D8
:1000A8000C9400000C9400000C9400000C940000C8
:1000B8000C9400000C9400000C9400000C940000B8
:1000C8000C9400000C9400000C9400000C940000A8
:1000D8000C9400000C9400000C9400001027E80316
:1000E80064000A0001000010000110000100686FA0
:1000F80075723A202564206D696E7574653A2025FD
:1001080064207365636F6E643A2025640D0A0000ED
:10011800F894EE27EFBBF1E0F5BFE5BFE09374007C
:10012800E0937500F8E1A895A4B7A77FA4BFF09362
:100138006000E09360008DE0A2E0BB27ED938A9514
:10014800E9F780E090E2A0E0B2E0ED930197E9F7EB
:100158008BBF8CBFE0E0EEBBEFEFEDBFE1E2EEBF9F
:10016800C0E0DAE00C940F01E4EAE093BC00E0910F
:10017800BC00E078E1F30E940003E091BC00E07865
:10018800E1F30E940703E091BC00E078E1F3E88125
:10019800E093BB00E4E8E093BC00E091BC00E078A9
:1001A800E1F3E4E9E093BC0034C01A9310E0E4EA18
:1001B800E093BC00E091BC00E078E1F30E9400030A
:1001C800E091BC00E078E1F30E940703E091BC00F5
:1001D800E078E1F3E4EAE093BC00E091BC00E07869
:1001E800E1F3E1EDE093BB00E4E8E093BC00E091CB
:1001F800BC00E078E1F3E4E8E093BC00E091BC00E7
:10020800E078E1F31091BB00E4E9E093BC00E12F52
:10021800188122960895E0E8E0936100E0E0E09319
:100228006100E093C000E8E0E093C100E6E0E093FD
:10023800C200E0E0E093C500E7E6E093C400E2E135
:10024800E093B800E0E0E093B900E4E0E093BC009C
:10025800E0E0EA93EA9388DFE1E0EA93E3E0EA93F7
:1002680083DFE2E0EA93E6E0EA937EDFE7E0EA9301
:10027800E3E0EA9379DFE0E00E940E03E093050AE9
:10028800E1E00E940E03E093040AE2E0EA938DDFC6
:10029800E093000AEF70E093010AE091000AE0732E
:1002A800E093020AF0E00E946003AAE0EA02F0018B
:1002B800E093020AE091010AA091020AEA0FE09392
:1002C800030AE6EFF0E0FA93EA93E091030A0E944A
:1002D8002903E091040A0E942903E091050A0E947B
:1002E80029038CE04DD12E96C6CFFFCFE091C000F8
:1002F800E072E1F3E881E093C60021960895EA816F
:10030800EA93F4DFA881B981ED91FD913196FE93CE
:10031800EE932396089526970E94760310E0AC8505
:10032800BD85E0E0F0E0ED93FC93EA89FB89319626
:10033800EA8BFB8B3197E4912E2FE03011F40C946B
:10034800BC02E12FE03039F4253211F411E002C08B
:100358000E942F030CC1E130A9F4253219F40E9440
:100368002F0304C112E040E000E02D3211F401E057
:10037800FEC02B3211F44BE2FAC0203211F440E2F5
:10038800F6C002C0E23039F450E013E0203311F433
:100398000068EDC004C0E33011F00C94BB022033B8
:1003A80010F02A3308F007C0AAE05A9F502DE22F18
:1003B800E0535E0FDCC0E22FE33649F40E943803B5
:1003C800E889F989A481AA930E943E03CFC0E33744
:1003D80041F40E9438030E9446030E94EB021E2F3C
:1003E8000AC0E03761F40E9438030E9446030E9465
:1003F800F5021E2F086002600F7730E035C0E43642
:1004080011F0E93611F4046002C0E53731F4E4EE86
:10041800F0E0EE83FF8315E00DC0E83511F40860C5
:1004280004C0E83711F00C94BA02EEEEF0E0EE8367
:10043800FF8314E002FF14C00E9438030E94500397
:10044800AB85AA233AF4EA85FB850E945C03EA8718
:10045800FB874DE2403011F01F5F01C00B7F04C0E5
:100468000E9438030E94500300FD11C0151778F44C
:1004780007FF08C002FF04C00B7F242F115001C0E2
:1004880020E301C020E20E942F035150EFCF312F0B
:1004980001FF17C03030A1F003FF06C0EE81FF81D5
:1004A8002591EE83FF8305C0AE81BF812D91AE8378
:1004B800BF830E942F03503009F051503150EACFCA
:1004C8004BC020E3EE81FF810E946D03E887F98726
:1004D800EE81FF813296EE83FF83E885F985AA8550
:1004E800BB85AE17BF0750F02F5FA885B985EA8591
:1004F800FB85EA1BFB0BEA87FB87EFCF2A3328F043
:1005080003FF02C0295F01C0295D04FD1AC0213321
:1005180020F4A885B985119709F409C0531710F07C
:1005280000FF01C013C020E207FF0BC020E30061F9
:1005380002FF07C00B7F4A930E943E03503009F028
:1005480051500E942F03503009F051503150A88566
:10055800B985129708F0B5CF00FF08C0503031F0C8
:100568005150E0E2EA930E943E03F8CF10E0DDCE5E
:10057800AC85BD850E9469030E947D036496089539
:10058800FF92F82E26971A930A93DE0114960E947A
:1005980058038D01E0E0EC83ED83EE83EF83DE0109
:1005A80018960E9458030E946903FA93EA931A93D3
:1005B8000A93E3E8F1E0FA93EA93FE013896FA9396
:1005C800EA93A9DE198108812896FF900895A991D8
:1005D800B991EE27FF276D91662311F03196FBCF75
:1005E8000895AA27BB27E991F9910590002011F0F9
:1005F8001196FBCFFD010895E0EDE093BB00E4E820
:10060800E093BC000895E981E093BB00E4E8E0933F
:10061800BC000895EA930E94D900E093000AEF70A5
:10062800E093010AE091000AE077E093020AF0E023
:100638000E946003AAE0EA02F001E093020AE09156
:10064800010AA091020AEA0F0895FF276627772773
:100658000E94710308952A93ED85FE85FA93EA9323
:10066800E989FA8909950895E889F9893497E88B21
:10067800F98B0895ED85FE85FA93EA93E989FA895D
:1006880009950895A889B98914960E946903EE838B
:10069800FF83FA93EA930895A889B98914960E946A
:1006A8006903EA87FB8708950024AF0DB01D0895FC
:1006B800F195E195F0400895F595E795F595E7955D
:1006C800F595E795F595E7950895ED91FC911197C6
:1006D80008950590F491E02D08957A936A93FA931A
:1006E800EA9308955A934A933A932A931A930A934A
:1006F80008955D814C813B812A8119810881089583
:00000001FF
